:0A00000075817F7401F58F02000E78
:10000B0002023FC229C2287400900010F090001128
:10001B00F0900012F0900013F0900014F074009028
:10002B000016F07401900017F07402900018F07431
:10003B0003900019F0740490001AF0740590001BE3
:10004B00F0740690001CF0740790001DF07408907B
:10005B00001EF0740990001FF0740A900020F074D9
:10006B000B900021F07400900031F0900032F09072
:10007B000033F0900034F0900035F0740290002FB4
:10008B00F07402900030F090003779FF7400F0A309
:10009B00D9FA90013679FF7400F0A3D9FA900237A0
:1000AB0079FF7400F0A3D9FA90033679CD7400F080
:1000BB00A3D9FA120EC57564FF7565FF7566FF75DA
:1000CB00460075470075710075680075720075699B
:1000DB0000C208C2097540007541007542007543A6
:1000EB0000754C00754D007570027548FF75490A17
:1000FB0085483C85493D754A7F754B01854A44854A
:10010B004B45755500D226C2C175A012C2B1C2B300
:10011B00C2B4C2B5C2B6C281C2B2C2841206AC129C
:10012B0006CB1206EA12070912082075597F755A79
:10013B007F755B7F755D00755E00755F001201EF6B
:10014B001205A712060212218C75730075740175C6
:10015B0072001216DA121F2A121F35D20FD22CC2BE
:10016B002E12238B12082012241D122549121F2A2E
:10017B00121F351208C3120B14120EE212154D1278
:10018B001565121CE5121CCA1223C002016C856096
:10019B0090C2A7C2C0D2C022856290D2A7C2C0D2E1
:1001AB00C022C285C281C2B2C284E56479081392AF
:1001BB0083C285D285D9F7D2810000C281E56579EA
:1001CB0008139283C285D285D9F7D2B20000C2B28E
:1001DB00E5667908139283C285D285D9F7D284005C
:1001EB0000C28422758790758922758DFC758BFCF6
:1001FB00759850C299C298758C38758A38753906BE
:10020B00753A04753B0590FF9C8582CA8583CB8527
:10021B0082CC8583CDC200C201D28CD2A9D2AF22AF
:10022B00783279320000D9FCD8F822780A790FD9C4
:10023B00FED8FA22C2AFC0E0C0D0E5F0C0E0E58244
:10024B00C0E0E583C0E0E575C0E0E8C0E0E9C0E0F0
:10025B00EAC0E0EBC0E01206EA1224F5122509D53C
:10026B0044107544FFD5450A854A44854B45D22336
:10027B00D22712243712246E121AFA12244D1203AB
:10028B00F512045312251D12248DD5392D753906FF
:10029B00B2033003091207281206940202AC1201B2
:1002AB00ADD53A16753A041211BF1201991201A37A
:1002BB00303307D53B04D2A0C233D0E0FBD0E0FAF9
:1002CB00D0E0F9D0E0F8D0E0F575D0E0F583D0E0E0
:1002DB00F582D0E0F5F0D0D0D0E0D2AF32E54FB41C
:1002EB00021130240ED287C282054DD2A2121F6793
:1002FB0002204C22E55575F001241084E5F0B40082
:10030B0014E54FB40006755680020385B4020675DA
:10031B00568002038522E55575F001241084E5F023
:10032B00B4000BE54FB4000675565002038522E569
:10033B005575F002241084E5F0B4000BE54FB400C2
:10034B000675562202038522E55575F004241084A8
:10035B00E5F0B4000BE54FB40006755610020385AB
:10036B0022E55575F008241084E5F0B4000BE54F39
:0E037B00B4000675560702038522200C0C30D4
:100389002409D2B6C280D2041211D7D21B85525089
:1003990022E55A75F01E84B4040302036CB4050304
:1003A900020353B4060302033AB40703020321B458
:1003B900080302032122E559B40F030203C95005BA
:1003C90074010203D7C3940F8556F0842401F552B2
:1003D90022E559B40F030203E4500574010203F244
:1003E900C3940F8556F0842401F55322D53C0302AA
:1003F9000422D53C03020422D53C03020422D53C45
:1004090003020422D53C03020422D53C0302042240
:10041900D53C03020422D53C0DD53D0A85483C85CF
:10042900493D054FD2013001201202E8301B0FD59A
:10043900500CC21B202007302404C2B6D280121DE2
:100449006E12039A1203BFC20122D53E030204743D
:10045900D53E03020474D53E03020474D53E03025B
:100469000474D53E03020474D53E0DD53F0A854870
:100479003E85493F054ED20030000B12049012050B
:10048900881203DAC20022201A0122D5500CC21A9E
:10049900202007302404C2B6D28022E55575F00227
:1004A900241084E5F0B40014E54EB40006755680B6
:1004B900020573B40214755680020573B4010BE585
:1004C9004EB4010675568002057322E55575F00490
:1004D900241084E5F0B4010BE54EB400227556787A
:1004E900020573B4020BE54EB40114755678020582
:1004F90073B4030BE54EB4020675567802057322F0
:10050900E55575F008241084E5F0B4010BE54EB407
:100519000022755630020573B4030BE54EB402147C
:10052900755630020573B4060BE54EB401067556CF
:100539003002057322E55575F010241084E5F0B4F6
:10054900010BE54EB40022755615020573B4060B6E
:10055900E54EB40114755615020573B40B0BE54E3F
:10056900B4020675561502057322200C0C302409B5
:10057900D2B6C280D2041211D7D21A85535022E5BD
:100589005A75F01E84B400030204D4B401030204B2
:10059900D4B40203020509B4030302053E227564BB
:1005A900F71202367564DF1202367564FF7565F756
:1005B9001202367565FD1202367565FF7566DF1222
:1005C90002367566FD12023675667F120236756649
:1005D900FF75647F1202367564FD1202367564FF79
:1005E9007565DF12023675657F1202367565FF750E
:1005F90066F71202367566FF227564F312023675C4
:1006090064CF1202367564FF7565F312023675659B
:10061900FC1202367565FF7566CF1202367566FCE7
:1006290012023675663F1202367566FF75643F120F
:1006390002367564FC1202367564FF7565CF1202C5
:100649003675653F1202367565FF7566F312023617
:100659007566FF227564001201AD7564001201AD63
:0E0669007564001201AD7564551201AD756423
:10067700001201AD7564001201AD7564001201AD81
:100687007566551201AD7565001201AD22E546B4D8
:10069700000505460206ACB4010505460206CB7502
:1006A700460002070974FE7908339283D285C28512
:1006B700D9F7C2B7D2B77908A2A133D2A6C2A6D9B1
:1006C700F7F56A2274FD7908339283D285C285D9FA
:1006D700F7C2B7D2B77908A2A133D2A6C2A6D9F773
:1006E700F56B2274FB7908339283D285C285D9F7DB
:1006F700C2B7D2B77908A2A133D2A6C2A6D9F7F555
:100707006C2274F77908339283D285C285D9F7C2F0
:10071700B7D2B77908A2A133D2A6C2A6D9F7F56D89
:1007270022E547B400050547020758B40105054708
:10073700020776B402050547020798B40305054783
:100747000207BAB4040505470207E4754700020823
:1007570002C2A3C286C2B0D2A57914D9FEC2A579B6
:1007670008C2A6D2A6A2A433D9F7C2A6F55D22D2A3
:10077700A3C286C2B0D2A57914D9FEC2A57908C290
:10078700A6D2A6A2A433D9F7C2A630280122F559CA
:1007970022C2A3D286C2B0D2A57914D9FEC2A57946
:1007A70008C2A6D2A6A2A433D9F7C2A6302801222E
:1007B700F55A22D2A3C286D2B0D2A57914D9FEC2E5
:1007C700A57908C2A6D2A6A2A433D9F7C2A6302813
:1007D700030207DDF55B30290122F55C22D2A3D2A3
:1007E70086C2B0D2A57914D9FEC2A57908C2A6D20D
:1007F700A6A2A433D9F7C2A6F55E22C2A3C286D2A7
:10080700B0D2A57914D9FEC2A57908C2A6D2A6A2EC
:10081700A433D9F7C2A6F55F2212084A1208581264
:10082700083C12086612087412088212089012080F
:10083700A11208B222E56C30E4012220E6012275FC
:100847006E0022E56C20E4012220E60122756E018C
:1008570022E56C20E4012230E60122756E0222E5D2
:100867006B30E3012220E50122756F0022E56B2042
:10087700E3012220E50122756F0122E56B20E301E8
:100887002230E50122756F0222E56D30E601222054
:10089700E50122740190002FF022E56D20E6012288
:1008A70020E50122740290002FF022E56D20E60179
:1008B7002230E50122740490002FF022E56F7017B3
:1008C700C22EC22DD20F1208DF120A1812094412C3
:1008D7000B0E1209EBD22C22302907900031E002CF
:1008E70008EBE55CB478030208F650030208F874D5
:1008F7007975F01784B4000C756700C2B1C2B3C232
:10090700B5C2B422B4010C756701D2B1C2B3C2B586
:10091700C2B422B4020C756702C2B1D2B3C2B5C267
:10092700B422B4030C756703C2B1C2B3D2B5C2B463
:1009370022756704C2B1C2B3C2B5D2B422E56775E6
:10094700F030A42568F56022E56BF430E009757195
:1009570001D22A1209F42230E109757100D22A1254
:1009670009F42230E209757102D22A1209F4223001
:10097700E609757103D22A1209F422E56AF430E018
:1009870009757106D22A1209F42230E10975710935
:10099700D22A1209F42230E20975710AD22A120901
:1009A700F42230E309757107D22A1209F42230E4E0
:1009B7000975710BD22A1209F42230E509757108FD
:1009C700D22A1209F42230E609757105D22A1209D2
:1009D700F42230E709757104D22A1209F422C22AD7
:0E09E7001209F422202A03D2A022C2A022E587
:1009F50071202A05C2E7F56922D2E7F56922900040
:100A050032E020E707C22AC2E7F57122D22AC2E7FF
:100A1500F57122302906120A03020A2712094F022C
:100A25000A27E571B4011075680412094475647FDD
:100A35007565FF7566FF22B40010756800120944DC
:100A45007564F77565FF7566FF22B4021075680851
:100A55001209447564DF7565FF7566FF22B40310DE
:100A650075680C1209447564FD7565FF7566FF228E
:100A7500B406107568181209447564FF7565DF754D
:100A850066FF22B409107568241209447564FF7560
:100A950065FF7566FD22B40A10756828120944754C
:100AA50064FF7565FF7566F722B4071075681C123B
:100AB50009447564FF7565FF7566DF22B40B107513
:100AC500682C1209447564FF7565FF75667F22B44D
:100AD50008107568201209447564FF75657F756691
:100AE500FF22B405107568141209447564FF756515
:100AF500FD7566FF22B4041075681012094475640B
:100B0500FF7565F77566FF2222E571120CEE22E589
:100B15006F7003D20F22E56EB40212D22CC22EC220
:100B25002D300F05120EB9C20F120CD122D20F2291
:100B3500E55EB43803020B3F5003790022B43C0351
:100B4500020B4A5003790122B44103020B555003AD
:100B5500790222B44503020B605003790322B44A9B
:100B650003020B6B5003790422B44E03020B76503B
:100B750003790522B45303020B815003790622B48D
:100B85005703020B8C5003790722B45C03020B97C1
:100B95005003790822B46003020BA250037909229D
:100BA500B46503020BAD5003790A22B46A03020B44
:100BB500B85003790B22790B22120B35E9900033DB
:100BC500F0120CCC120EB922900033E0F575120B21
:100BD50035E9B57503020BF7E55EB43404120BBEB7
:100BE500225003020BF7B46B03020BF75004120BF0
:100BF500BE22E56BF430E00E200E51D20E790112C3
:100C05000CCC120EB92230E10E200E40D20E790026
:100C1500120CCC120EB92230E20E200E2FD20E7914
:100C250002120CCC120EB92230E60E200E1ED20E88
:100C35007903120CCC120EB922E56AF430E00E20CD
:100C45000E0AD20E7906120CCC120EB92230E10E24
:100C5500200E70D20E7909120CCC120EB92230E298
:100C65000E200E5FD20E790A120CCC120EB922306C
:100C7500E30E200E4ED20E7907120CCC120EB922BD
:100C850030E40E200E3DD20E790B120CCC120EB9AB
:100C95002230E50E200E2CD20E7908120CCC120E45
:100CA500B92230E60E200E1BD20E7905120CCC129D
:100CB5000EB92230E70E200E0AD20E7904120CCCA2
:100CC500120EB922C20E228969897122302911902A
:100CD5000032E0C2E7B5710122D20FF571020EB9FB
:100CE500020BCDE571120CEE22B4010A75647F7515
:100CF50065FF7566FF22B4000A7564F77565FF75B3
:100D050066FF22B4020A7564DF7565FF7566FF220A
:100D1500B4030A7564FD7565FF7566FF22B4060A9E
:100D25007564FF7565DF7566FF22B4090A7564FF92
:100D35007565FF7566FD22B40A0A7564FF7565FF62
:0C0D45007566F722B4070A7564FF756537
:100D5100FF7566DF22B40B0A7564FF7565FF756662
:100D61007F22B4080A7564FF75657F7566FF22B43A
:100D7100050A7564FF7565FD7566FF22B4040A7581
:100D810064FF7565F77566FF2222B4010A75643F39
:100D91007565FF7566FF22B4000A7564F37565FF1A
:100DA1007566FF22B4020A7564CF7565FF7566FF2B
:100DB10022B4030A7564FC7565FF7566FF22B406EB
:100DC1000A7564FF7565CF7566FF22B4090A7564FB
:100DD100FF7565FF7566FC22B40A0A7564FF7565C7
:100DE100FF7566F322B4070A7564FF7565FF7566C2
:100DF100CF22B40B0A7564FF7565FF75663F22B497
:100E0100080A7564FF75653F7566FF22B4050A75AA
:100E110064FF7565FC7566FF22B4040A7564FF758D
:100E210065F37566FF2222B40109E564C2E7D2E6E3
:100E3100F56422B40009E564C2E3D2E2F56422B4A8
:100E41000209E564C2E5D2E4F56422B40309E5646C
:100E5100C2E1D2E0F56422B40609E565C2E5D2E457
:100E6100F56522B40909E566C2E1D2E0F56622B46E
:100E71000A09E566C2E3D2E2F56622B40709E5662E
:100E8100C2E5D2E4F56622B40B09E566C2E7D2E613
:100E9100F56622B40809E565C2E7D2E6F56522B434
:100EA1000509E565C2E1D2E0F56522B40409E5650D
:100EB100C2E3D2E2F5652222120EC5121104E571D8
:100EC100120E2822790C90002205A2900016E0A3B0
:100ED10020E70605A2F0A305A2D9F305A27480F0CC
:100EE10022E56F700122E56EB40116D22CC22F12D9
:100EF10017131216F6202E09120F03120FCD120E20
:100F0100C522E56BF430E00D200D4CD20D90001799
:100F1100E0B2E7F02230E10D200D3CD20D90001639
:100F2100E0B2E7F02230E20D200D2CD20D90001836
:100F3100E0B2E7F02230E60D200D1CD20D90001931
:100F4100E0B2E7F022E56AF430E00D200D09D20DA0
:100F510090001CE0B2E7F02230E10D200D6DD20DC2
:100F610090001FE0B2E7F02230E20D200D5DD20DBE
:100F7100900020E0B2E7F02230E30D200D4DD20DBC
:100F810090001DE0B2E7F02230E40D200D3DD20DBE
:100F9100900021E0B2E7F02230E50D200D2DD20DB9
:100FA10090001EE0B2E7F02230E60D200D1DD20DBB
:100FB10090001BE0B2E7F02230E70D200D0DD20DBD
:100FC10090001AE0B2E7F022C20D2222900017E051
:100FD10020E70BE564C2E7C2E6F564020FE7E564CA
:100FE100D2E7D2E6F564900016E020E70BE564C293
:100FF100E3C2E2F564021001E564D2E3D2E2F564F2
:10100100900018E020E70BE564C2E5C2E4F5640254
:10101100101BE564D2E5D2E4F564900019E020E705
:101021000BE564C2E1C2E0F564021035E564D2E18A
:10103100D2E0F56490001CE020E70BE565C2E5C253
:10104100E4F56502104FE565D2E5D2E4F56590005F
:101051001FE020E70BE566C2E1C2E0F56602106918
:02106100E56642
:10106300D2E1D2E0F566900020E020E70BE566C20E
:10107300E3C2E2F566021083E566D2E3D2E2F566E7
:1010830090001DE020E70BE566C2E5C2E4F56602C9
:10109300109DE566D2E5D2E4F566900021E020E7F5
:1010A3000BE566C2E7C2E6F5660210B7E566D2E76E
:1010B300D2E6F56690001EE020E70BE565C2E7C2C5
:1010C300E6F5650210D1E565D2E7D2E6F565900055
:1010D3001BE020E70BE565C2E1C2E0F5650210EB1A
:1010E300E565D2E1D2E0F56590001AE020E709E575
:1010F30065C2E3C2E2F56522E565D2E3D2E2F565B6
:10110300227564FF7565FF7566FF900022E0FAE0C3
:10111300F92571C39AB40C0302112350030211265B
:10112300C3940C12112FA3E930E7E422B40109E5BB
:1011330064C2E7C2E6F56422B40009E564C2E3C20F
:10114300E2F56422B40209E564C2E5C2E4F564226F
:10115300B40309E564C2E1C2E0F56422B40609E51B
:1011630065C2E5C2E4F56522B40909E566C2E1C2D8
:10117300E0F56622B40A09E566C2E3C2E2F5662237
:10118300B40709E566C2E5C2E4F56622B40B09E5D6
:1011930066C2E7C2E6F56622B40809E565C2E7C29E
:1011A300E6F56522B40509E565C2E1C2E0F565220D
:1011B300B40408E565C2E3C2E2F56522E56FB40154
:1011C30009E56C30E501221214CE22E56FB4020367
:1011D30012152A2230040DC204202008E56FB40240
:1011E300031214CE22E55DB402030211F250037917
:1011F3000022B406030211FD5003790122B40A034D
:101203000212085003790222B40F0302121350038F
:10121300790322B4130302121E5003790422B41873
:10122300030212295003790522B41D03021234501C
:1012330003790622B4210302123F5003790722B433
:10124300250302124A5003790822B42A03021255D5
:101253005003790922B42E030212605003790A2243
:10126300B4330302126B5003790B22790B22E55D31
:10127300B4370302127B5003790022B43C030212F9
:10128300865003790122B44003021291500379027C
:1012930022B4450302129C5003790322B44903028A
:1012A30012A75003790422B44E030212B2500379F9
:1012B3000522B452030212BD5003790622B4570328
:1012C3000212C85003790722B45B030212D35003FE
:1012D300790822B460030212DE5003790922B46450
:1012E300030212E95003790A22B468030212F4508C
:1012F30003790B22790B22E55DB46D0302130450CD
:1013030003790022B4710302130F5003790122B44D
:10131300760302131A5003790222B47A03021325C7
:101323005003790322B47E0302133050037904225D
:10133300B4830302133B5003790522B487030213DA
:10134300465003790622B48C0302135150037907E4
:1013530022B4900302135C5003790822B49503026C
:1013630013675003790922B4990302137250037966
:101373000A22B49E0302137D5003790B22790B22B8
:10138300E55DB4A20302138D5003790022B4A703D1
:101393000213985003790122B4AB030213A3500341
:1013A300790222B4B0030213AE5003790322B4B41A
:1013B300030213B95003790422B4B9030213C450CE
:1013C30003790522B4BD030213CF5003790622B477
:0E13D300C1030213DA5003790722B4C60302E5
:1013E10013E55003790822B4CA030213F0500379BC
:1013F1000922B4CF030213FB5003790A22B4D403A8
:101401000214065003790B22790B22E55DB4D8034F
:101411000214165003790022B4DC03021421500394
:10142100790122B4E10302142C5003790222B4E5BC
:10143100030214375003790322B4EA030214425021
:1014410003790422B4EE0302144D5003790522B44A
:10145100F3030214585003790622B4F7030214630C
:101461005003790722B4FC0302146E500379082259
:10147100B4FE030214795003790922790A22E55D49
:10148100B4330302148950091211E889757400FB01
:1014910022B4680302149A500912127189757401F9
:1014A100FB22B49E030214AB50091212FA8975741F
:1014B10002FB22B4D4030214BC50091213838975B0
:1014C1007403FB2212140C89757404FB2212147F1D
:1014D1007A00900022E020E70DB575030214E85070
:1014E10006A3FA0214D6EA2571F9BB0424B40A034F
:1014F100021512401C7A00900022E020E70D2571B0
:10150100B40A06E0FAA30214FB40F8EA25710215B9
:1015110013E975F004A4F9EB75F030A4FAE92AF5A2
:1015210060EB1208FC12153822900036E0F560EBF2
:101531001208FC12153822E56F6010E560B56101F3
:1015410022856061C2A0D233753B0522E56F70012F
:1015510022E56EB4000DC22EC22D1219FF121660C3
:1015610012159722E56F700122E56EB4011512196B
:10157100FF30300F1216DA120F03120FCD120EC503
:10158100C23022B4020F1219FF3031091216DA12D9
:101591000EB9C2312222202C0122E573120D8BE5F6
:1015A10074120E28C22CE56F700122E56EB400069C
:1015B100302F031216DA22E56BF430E114E572C222
:1015C100E0C2E1C2E2C2E3F572757300D22CD22F00
:1015D1002230E214E572D2E0C2E1C2E2C2E3F57266
:1015E100757302D22CD22F22E56AF430E114E57230
:1015F100D2E0C2E1D2E2C2E3F572757309D22CD214
:101601002F2230E314E572C2E0C2E1D2E2C2E3F577
:1016110072757307D22CD22F2230E414E572C2E026
:10162100D2E1D2E2C2E3F57275730BD22CD22F2232
:1016310030E614E572D2E0D2E1C2E2C2E3F572759E
:101641007305D22CD22F2230E714E572C2E0D2E129
:10165100C2E2C2E3F572757304D22CD22F2222E5C5
:101661006BF430E014E572C2E4C2E5C2E6C2E7F50C
:1016710072757401D22CD22F2230E614E572D2E4B5
:10168100C2E5C2E6C2E7F572757403D22CD22F22ED
:10169100E56AF430E014E572C2E4D2E5C2E6C2E7DD
:1016A100F572757406D22CD22F2230E514E572D270
:1016B100E4D2E5C2E6C2E7F572757408D22CD22FE6
:1016C1002230E214E572C2E4C2E5D2E6C2E7F57265
:1016D10075740AD22CD22F2222E572C2E0C2E1C275
:1016E100E2C2E3C4B4040712213F120EC522122143
:1016F1006A120EC522E56C30E303C22B22202B11A6
:10170100D22B202D05D22ED22D22C22E12210FC274
:101711002D22202E0122E572C2E4C2E5D2E6C2E703
:10172100F57275740A1215B812159722900034E0FB
:10173100F5751219FFE9B57503021757E55FB43462
:10174100041219FF225003021757B454030217570A
:0E17510050041219FF221215B822E55FB437BA
:10175F000302176550077401900035F022B43C0363
:10176F0002177450077402900035F022B440030240
:10177F00178350077403900035F022B44503021706
:10178F009250077404900035F022B449030217A158
:10179F0050077405900035F022B44E030217B05075
:1017AF00077406900035F022B452030217BF50079A
:1017BF007407900035F02222E55FB457030217D16A
:1017CF0050077401900035F022B45B030217E0500C
:1017DF00077402900035F022B460030217EF500730
:1017EF007403900035F022B464030217FE5007749F
:1017FF0004900035F022B4680302180D50077405E9
:10180F00900035F022B46D0302181C500774069037
:10181F000035F022B4710302182B500774079000A3
:10182F0035F02222E55FB4760302183D50077401AC
:10183F00900035F022B47A0302184C5007740290CE
:10184F000035F022B47E0302185B5007740390003A
:10185F0035F022B4830302186A50077404900035E0
:10186F00F022B4870302187950077405900035F001
:10187F0022B48C0302188850077406900035F022AA
:10188F00B4900302189750077407900035F0222286
:10189F00E55FB495030218A950077401900035F065
:1018AF0022B499030218B850077402900035F02241
:1018BF00B49E030218C750077403900035F022B48A
:1018CF00A2030218D650077404900035F022B4A773
:1018DF00030218E550077405900035F022B4AB03EE
:1018EF000218F450077406900035F022B4B00302CA
:1018FF00190350077407900035F02222E55FB4B446
:10190F000302191550077401900035F022B4B90382
:10191F0002192450077402900035F022B4BD03025F
:10192F00193350077403900035F022B4C103021924
:10193F004250077404900035F022B4C603021951C7
:10194F0050077405900035F022B4CA030219605095
:10195F00077406900035F022B4CF0302196F5007B9
:10196F007407900035F02222E55FB4330122500155
:10197F0022B45203021988501312175BE572C2E4A6
:10198F00C2E5C2E6C2E7F57275740122B4710302B3
:10199F0019A350131217C7E572D2E4C2E5C2E6C20B
:1019AF00E7F57275740322B490030219BE50131237
:1019BF001833E572C2E4D2E5C2E6C2E7F572757478
:1019CF000622B4B0030219D9501312189FE572D230
:1019DF00E4D2E5C2E6C2E7F5727574082212190B5C
:1019EF00E572C2E4C2E5D2E6C2E7F57275740A2267
:1019FF00121977900034E0F576900035E0B5760E49
:101A0F00E56F700122E56EB400031215B822D22FD4
:101A1F00900035E0900034F0B40103021A2F5016F5
:101A2F00E572C2E0C2E1C2E2C2E3F572757300D2A1
:101A3F002CD231D23022B40203021A4D5016E57265
:101A4F00D2E0C2E1C2E2C2E3F572757302D22CD2C8
:101A5F0031D23022B40303021A6B5016E572C2E082
:101A6F00D2E1C2E2C2E3F572757304D22CD231D245
:101A7F003022B40403021A895016E572D2E0D2E183
:101A8F00C2E2C2E3F572757305D22CD231D2302285
:101A9F00B40503021AA75016E572C2E0C2E1D2E202
:101AAF00C2E3F572757307D22CD231D23022B4064D
:101ABF0003021AC55016E572D2E0C2E1D2E2C2E3C8
:0E1ACF00F572757309D22CD231D23022B407D1
:101ADD0003021AE35016E572C2E0D2E1D2E2C2E38C
:101AED00F57275730BD22CD231D230222230231ADB
:101AFD00054C121C93121B36121B6F121B1A121B54
:101B0D005E121C41121CA7121D0BC22322E54C753F
:101B1D00F018246084E5F0B40C06202402C2822261
:101B2D00B40005202402D28222E54C75F006246013
:101B3D0084E5F0B4030C202408D287121F6702201D
:101B4D004C22B4000B202408C287121F6702204CC0
:101B5D0022E54CB4600B754C00202405C2A2121F67
:101B6D00402220240BE54CB4000122B40302D2A282
:101B7D0022E54C75F030246084E5F0B4000975570A
:101B8D0008756360021C7E22E54C75F01824608494
:101B9D00E5F0B4000975570F756360021C7E22E5F0
:101BAD004C75F00C246084E5F0B4000975571E7572
:101BBD006360021C7E22E54C75F006246084E5F01E
:101BCD00B4000975573C756360021C7E22E54C75A7
:101BDD00F003246084E5F0B40009755778756360EF
:101BED00021C7E22E54C75F020246084E5F0B400E3
:101BFD000675570A021C7E22E54C75F01024608490
:101C0D00E5F0B40006755714021C7E22E54C75F004
:101C1D0008246084E5F0B40006755728021C7E2266
:101C2D00E54C75F004246084E5F0B400067557505A
:101C3D00021C7E22E55A75F01E84B40003021C2D91
:101C4D00B40103021C19B40203021C05B403030200
:101C5D001BF1B40403021B7EB40503021B95B406ED
:101C6D0003021BACB40703021BC3B40803021BDA47
:101C7D0022200C0C202409D2B6C280D2041211D716
:101C8D00D21C85545122201C0122D5510CC21C207E
:101C9D002007202404C2B6D28022E559B40F0302D6
:101CAD001CB150057401021CBFC3940F8557F084FD
:101CBD002401F554E557B4800375540122E5597597
:101CCD00F00484B40005D20CC22022B43F05C20C2E
:101CDD00D22022C20CC22022E55BB4A003021CF963
:101CED00500A12236475F002A4021D08B4C8030241
:101CFD001D0750061223EF021D0822F56222E55B37
:101D0D00B4C803021D154032B4FA03021D1D502B39
:101D1D00E54C75F003246084E5F0B4001DE54C75C9
:101D2D00F060246084E5F0FAC374609A75F0028463
:101D3D00F5F07405A4202402F56222E54C75F0033C
:101D4D00246084E5F0B40018E54C75F060246084DF
:101D5D00E5F075F00284F5F07405A4202402F56217
:101D6D0022E55BB4C803021D784019B4FA03021DC5
:101D7D008050127420C3954D75F008A412235B306A
:101D8D002402F56222E54D75F008A412235B302480
:101D9D0002F56222202406E54CFB021DCCE54D75B3
:101DAD00F003A4FB021DCC20240EE54C75F003843A
:101DBD0075F002A4FB021DCCE54D75F002A4FB8568
:101DCD00823285833375340075350078328B3675E4
:101DDD0037007936122278868208868322E572C210
:101DED00E0C2E1C2E2C2E3C4B40004121E1222B486
:101DFD000104121E4A22B40204121E8222B40304EC
:101E0D00121EBA2222E572C2E4C2E5C2E6C2E7B4EE
:101E1D0000049025B322B401049025BF22B402041E
:101E2D009025CB22B403049025D722B40404902529
:101E3D00E322B405049025EF229025FB22E572C222
:0E1E4D00E4C2E5C2E6C2E7B400049026072214
:101E5B00B4010490261322B4020490261F22B4036B
:101E6B000490262B22B4040490263722B405049048
:101E7B0026432290264F22E572C2E4C2E5C2E6C297
:101E8B00E7B4000490265B22B4010490266722B4C9
:101E9B00020490267322B4030490267F22B4040418
:101EAB0090268B22B40504902697229026A322E538
:101EBB0072C2E4C2E5C2E6C2E7B400049026AF22C8
:101ECB00B401049026BB22B402049026C722B403AB
:101EDB00049026D322B404049026DF22B405049088
:101EEB0026EB229026F722E572C2E4C2E5C2E6C2D7
:101EFB00E7B4000490000022B4010490000C22B45B
:101F0B00020490001822B4030490002422B40404A9
:101F1B0090003022B4050490003C2290004822E54A
:101F2B006D30E403C22822D22822E56B30E403C2D1
:101F3B002922D229220570121F4D121F59900030F1
:101F4B00F02290002FE004B5700375700122900011
:101F5B002FE0B5700122400122F57022202822903B
:101F6B00002FE0B40412121F9E121DA1E559F0A31D
:101F7B00E55AF0A3E55BF022B40203021FB902207D
:101F8B0007121F9E121DA1E0F559A3E0F55AA3E01D
:101F9B00F55B22E570B4010490003722B402049083
:101FAB00009A22B403049000FD2290016022E57098
:101FBB00B40123900037121DA1E559F0A3E55AF0A7
:101FCB00A3E55BF09000FD121DA1E559F0A3E55AC6
:101FDB00F0A3E55BF022B4022290009A121DA1E55A
:101FEB0059F0A3E55AF0A3E55BF0900160121DA137
:101FFB00E559F0A3E55AF0A3E55BF0229000371208
:10200B001DA1E559F0A3E55AF0A3E55BF090009A0A
:10201B00121DA1E559F0A3E55AF0A3E55BF0900082
:10202B00FD121DA1E559F0A3E55AF0A3E55BF09075
:10203B000160121DA1E559F0A3E55AF0A3E55BF091
:10204B002220291E90002FE0B4040E122081121DB5
:10205B00B4E55CF0A3E569F022B4020302209C0214
:10206B0020DA122081121DB4E0F9A3E0900032F0C7
:10207B00E9900031F022E570B401049001C322B461
:10208B00020490020522B4030490024722900289B5
:10209B0022E570B4011B9001C3121DB4E55CF0A3E3
:1020AB00E569F0900247121DB4E55CF0A3E569F019
:1020BB0022B4021A900205121DB4E55CF0A3E56987
:1020CB00F0900289121DB4E55CF0A3E569F0229053
:1020DB0001C3121DB4E55CF0A3E569F09002051293
:1020EB001DB4E55CF0A3E569F0900247121DB4E561
:1020FB005CF0A3E569F0900289121DB4E55CF0A3D6
:10210B00E569F022C2AF790C90001605A2121EF2FF
:10211B0005A2122123D2AF22E0A343D20205A2F0E3
:10212B00A375D25275D2A2E5D220E0FB53D2FD05A6
:10213B00A2D9E522C2AF790C121EF205A2900016AD
:10214B0005A2122153D2AF2243D202438E20E0A329
:10215B0053D2FD538EDF05A2F0A305A2D9EA22C20A
:10216B00AF790C7B00121DEA05A290001605A21296
:10217B002180D2AF22EB9305A2F0A305A20BD9F5D8
:10218B0022E56BF430E163E56AF430E45D7405122B
:10219B000CEE1202361202361202361202361202FE
:1021AB0036120236120236C2AF1221F61222081272
:1021BB0022181222281222381222481222581222D6
:0F21CB0068D2AF120236120236120236120236F4
:1021DA001202361202361202361202361202361271
:1021EA00023612023612023612023622790C7B00AD
:1021FA009025A705A290001605A212218022790C2B
:10220A0090001605A290000005A212212322790C43
:10221A0090001605A290000C05A212212322790C27
:10222A0090001605A290001805A212212322790C0B
:10223A0090001605A290002405A212212322790CEF
:10224A0090001605A290003005A212212322790CD3
:10225A0090001605A290003C05A212212322790CB7
:10226A0090001605A290004805A212212322E62713
:10227A00F5270809E637F528782722C3E697F527D0
:10228A000809E697F52878272286278729080986E4
:10229A0028872A122318782C22862C08862D08864D
:1022AA002E08862F872909872A1222BB7827792E9A
:1022BA00227530007531101222FD1222CE1222F13F
:1022CA00D531F422C3E52E9529E52F952AE53094D8
:1022DA0000500122E52E9529F52EE52F952AF52F96
:1022EA00E5309400F53022B3E52733F527E52833A6
:1022FA00F52822C3E52C33F52CE52D33F52DE52EF3
:10230A0033F52EE52F33F52FE53033F53022E52767
:10231A008529F0A4F52C85F02DE528852AF0A4F569
:10232A002E85F02FE5288529F0A4252DF52DE52EFB
:10233A0035F0F52EE52F3400F52FE527852AF0A490
:10234A00252DF52DE52E35F0F52EE52F3400F52F48
:10235A0022B4F00122400274F022B4780122400231
:10236A00747822B43001224002743022900010E0C6
:10237A0004B410027400F0900000A98229F582E0EA
:10238A0022900014E0FA900011E004B40F0274FFE6
:10239A00F0902587932A900014F0900013E004B47B
:1023AA0010027400F0F9900014E0FA900000E5823F
:1023BA0029F582EAF022900014E0FA900012E00473
:1023CA00B4110274FFF0902596932A900014F0122B
:1023DA0023A42212237654016008122376541F2460
:1023EA006022747F2212237675F0058412236D24ED
:1023FA0030221223765401600D12237675F005847B
:10240A0012236D24302212237675F0058412236D6F
:10241A00246022E56C20E210D22430320FC282D22C
:10242A0087C2B6D280C23222C224D23222300912E4
:10243A000542E542B4FF0B0543E543B4FF04C20875
:10244A00C209220540E540B4FF190541E541B4FF40
:10245A00127540FF7541FF753CFF753DFF85404889
:10246A0085414922E56C30E103C20A22200A13D2CF
:10247A000A300906C2091225662275420075430010
:10248A00D20922E56C30E003C20B22200B48D20BA2
:10249A00302404C287D282E555240275F00284E50D
:1024AA00F0B40018854048854149754000754100DF
:1024BA0085483C85493D85483E85493F754F0075AD
:0124CA004EC3
:1024CB0000054D05551224E1D200D201302406122D
:1024DB001F6702204C22E555B4100E755500754D43
:1024EB0000302405C2A2121F4022E56C30E703C264
:1024FB000622200608D206D226D2B6C2A222E56B4D
:10250B0030E703C20722200708D207D226D2B6C271
:10251B00A2222024012220260122754000754100B1
:10252B0085483C85493D85483E85493F7555007535
:10253B004F00754E00754D00757001C22622302478
:10254B00012220260122754200754300854A4485ED
:10255B004B45754C00757001C2262285423285436E
:10256B003375340075350078327536187537007948
:10257B00361222A3864A08E604F54B2203002C0CE4
:10258B0001057E2133E6FF0B4D68146405150D5ACA
:10259B004B1B26351E1A96114042C8D5000102036B
:1025AB000405060708090A0B008102830405860748
:1025BB0088098A0B008182830485860788898A8B28
:1025CB00008182830485860788098A8B0081828338
:1025DB000485860788898A0B008182830485068798
:1025EB0088898A0B008182838405868788890A8B78
:1025FB00008182030485860788090A8B0081020308
:10260B008405860708898A0B0081020384058607E7
:10261B0008890A8B008182038485860788898A8BC7
:10262B00008182038485860788098A8B0081820357
:10263B008485860788890A8B0081820384850687B7
:10264B0088890A8B008182038405060788890A8B97
:10265B00008102038405860788090A8B0001820327
:10266B008405860708890A8B008102830485060787
:10267B0088098A0B008102038405068708098A0BE7
:10268B00008102830405860788090A8B0081028377
:10269B000485068708890A8B0081028384058607D7
:1026AB0088890A8B000182830405860708890A8BB7
:1026BB00008102038405060708898A0B0001820347
:1026CB008485860708898A8B000182830405860727
:1026DB0008898A0B008102830405860708890A8B07
:1026EB00008102030485060708098A0B0001820397
:1026FB000485060788090A8B464C414D45205441F9
:10270B004D45204D414348494E45204555524F209C
:10271B005241434B2056455253494F4E202D2032A8
:10272B003031302056455253494F4E20312E3033E5
:0D273B0020286329627920616D7065726548
:00000001FF
